:1000000012C087C0189518951895189518951895C9
:100010001895189518951895189518951895189578
:100020001895189518958FE58DBFC0E4E0E44E2E25
:1000300084E08EBFD4E0F4E05F2EEEEFF3E0A0E6C4
:10004000B0E088278D933197E9F769D4662488E773
:1000500081BB86E884BB80E082BB80E085BB929A4E
:10006000969A789480E080936A003FD48CE09FD485
:10007000ECE3FBE032D4E1E0F0E048D434D4ECE44B
:10008000FBE02BD484EF91E0BED4E2E5FBE025D485
:1000900084EF91E0B8D4E8E5FBE01FD48AEF90E06C
:1000A000B2D4EAE5FBE019D48AEF90E0ACD4ECE5F9
:1000B000FBE013D48AEF90E0A6D4EEE5FBE00DD48C
:1000C0008AEF90E0A0D4E0E6FBE007D48AEF90E06E
:1000D0009AD4E2E6FBE001D48AEF90E094D4E4E61F
:1000E000FBE0FBD38AEF90E08ED4E6E6FBE0F5D3AD
:1000F000E3E0F0E00BD4F9D3E8E6FBE0EED38BB716
:1001000080648BBF85B78F7D806A85BF8895F4CF6B
:10011000A9CF0F921F922F923F924F925F927F92A0
:10012000AF92BF920F931F932F933F934F935F9381
:100130006F937F938F939F93AF93BF93CF93DF93EF
:10014000EF93FF938FB78F938BB78F7B8BBF84E633
:1001500090E059D40027BB27A3E38C9184FB0EF4D5
:1001600001E040E0041709F001C01CD10027BB27C3
:10017000A0E38C9182FB0EF401E040E0041709F04B
:100180002BC0969888E290E03ED4A99AAA9A8AE079
:1001900090E039D4AA988AE090E035D4A998AA9A38
:1001A0008AE090E030D4AA980027BB27A0E38C9186
:1001B00087FB0EF401E040E0041709F001C029D0EC
:1001C0000027BB27A0E38C9187FB0EF401E041E000
:1001D000041709F001C045D18F918FBFFF91EF91B6
:1001E000DF91CF91BF91AF919F918F917F916F914F
:1001F0005F914F913F912F911F910F91BF90AF90C1
:100200007F905F904F903F902F901F900F90189588
:1002100008956BD38FE711E077D3E8E7FBE05DD378
:1002200080E0809369000027BB27A3E38C9180FBCB
:100230000EF401E040E0041709F005C0A9E6B0E0C3
:100240008C918F5F8C930027BB27A0E38C9181FB5F
:100250000EF401E040E0041709F005C0A9E6B0E0A3
:100260008C918E5F8C930027BB27A0E38C9180FB41
:100270000EF401E040E0041709F005C0A9E6B0E083
:100280008C918C5F8C930027BB27A3E38C9185FB1B
:100290000EF401E040E0041709F005C0A9E6B0E063
:1002A0008C91885F8C93009169000A3008F003C03C
:1002B000EAE5FBE012D3A8E2B4E0E9E6F0E0D3D34C
:1002C00004D311D381E080936100009161000F306D
:1002D00010F009F04AC080E08093600080E08093D5
:1002E000620000916200073010F009F01FC0A0E624
:1002F000B0E00C9142E0049F0C9200916000BB279B
:10030000A3E38C9183FB882780F9482F040FA0E694
:10031000B0E00C93AA9A8AE090E075D3AA98A2E67E
:10032000B0E08C918F5F8C9308F4DBCF0091690073
:100330004FE0049FA3E6B0E00C920091630040916F
:100340006100040FA3E6B0E00C93A3E6B0E0EC91EB
:10035000FF27A0E6B0E091E07BE7D8D3A1E6B0E0CC
:100360008C918F5F8C9308F4B0CF84E690E04BD3F0
:10037000969A8AEF8093640081E080936600B3D2FE
:10038000E6E8FBE0AAD27BD20027BB27A0E38C9152
:1003900082FB0EF401E040E0041709F001C0F4CF45
:1003A000A4D20895A2D2E4E9FBE097D29CD2ECE378
:1003B000FBE093D20027BB27A3E38C9184FB0EF4D0
:1003C00001E041E0041709F001C04AC081E08093D8
:1003D000610081E090E0A7E6B0E08D939C93A7E6F2
:1003E000B0E00D911C910A3F50E0150710F009F0A4
:1003F0000EC0A7E6B0E0ED91FC91A1E6B0E091E07F
:100400007BE784D3A7E6B0E059D208F4E8CF969A08
:100410008AEF8093640082E08093660066D2ECE30A
:10042000FBE05BD260D2E2EAFBE057D228D20027A1
:10043000BB27A0E38C9182FB0EF401E040E004179F
:1004400009F001C0F4CF0027BB27A3E38C9184FB04
:100450000EF401E040E0041709F001C0E8DF45D2E6
:10046000089543D28FE711E04FD2E2EBFBE035D2A3
:100470003AD2ECE3FBE031D2E1E0F0E047D281E0B8
:1004800080936100009161000F3010F009F0A8C165
:1004900080E08093600080E08093620000916200C1
:1004A000073010F009F01CC0A0E6B0E00C9142E06B
:1004B000049F0C9200916000BB27A3E38C9183FB07
:1004C000882780F9482F040FA0E6B0E00C93AA9A81
:1004D000AA98A2E6B0E08C918F5F8C9308F4DECFEF
:1004E000A1E6B0E0EC91FF27A5E6B0E091E01FD3D4
:1004F0004091650000916000041709F401C001C03B
:1005000068C1009161004FE0040FA3E6B0E00C93D6
:10051000A3E6B0E0EC91FF27A5E6B0E091E007D3B9
:100520004091650000916000041709F401C001C00A
:1005300050C1009161004EE1040FA3E6B0E00C93BE
:10054000A3E6B0E0EC91FF27A5E6B0E091E0EFD2A2
:100550004091650000916000041709F401C001C0DA
:1005600038C1009161004DE2040FA3E6B0E00C93A6
:10057000A3E6B0E0EC91FF27A5E6B0E091E0D7D28A
:100580004091650000916000041709F401C001C0AA
:1005900020C1009161004CE3040FA3E6B0E00C938E
:1005A000A3E6B0E0EC91FF27A5E6B0E091E0BFD272
:1005B0004091650000916000041709F401C001C07A
:1005C00008C1009161004BE4040FA3E6B0E00C9376
:1005D000A3E6B0E0EC91FF27A5E6B0E091E0A7D25A
:1005E0004091650000916000041709F401C001C04A
:1005F000F0C0009161004AE5040FA3E6B0E00C935F
:10060000A3E6B0E0EC91FF27A5E6B0E091E08FD241
:100610004091650000916000041709F401C001C019
:10062000D8C00091610049E6040FA3E6B0E00C9346
:10063000A3E6B0E0EC91FF27A5E6B0E091E077D229
:100640004091650000916000041709F401C001C0E9
:10065000C0C00091610048E7040FA3E6B0E00C932E
:10066000A3E6B0E0EC91FF27A5E6B0E091E05FD211
:100670004091650000916000041709F401C001C0B9
:10068000A8C00091610047E8040FA3E6B0E00C9316
:10069000A3E6B0E0EC91FF27A5E6B0E091E047D2F9
:1006A0004091650000916000041709F401C001C089
:1006B00090C00091610046E9040FA3E6B0E00C93FE
:1006C000A3E6B0E0EC91FF27A5E6B0E091E02FD2E1
:1006D0004091650000916000041709F401C001C059
:1006E00078C00091610045EA040FA3E6B0E00C93E6
:1006F000A3E6B0E0EC91FF27A5E6B0E091E017D2C9
:100700004091650000916000041709F401C001C028
:1007100060C00091610044EB040FA3E6B0E00C93CD
:10072000A3E6B0E0EC91FF27A5E6B0E091E0FFD1B1
:100730004091650000916000041709F401C001C0F8
:1007400048C00091610043EC040FA3E6B0E00C93B5
:10075000A3E6B0E0EC91FF27A5E6B0E091E0E7D199
:100760004091650000916000041709F401C001C0C8
:1007700030C00091610042ED040FA3E6B0E00C939D
:10078000A3E6B0E0EC91FF27A5E6B0E091E0CFD181
:100790004091650000916000041709F401C001C098
:1007A00018C00091610041EE040FA3E6B0E00C9385
:1007B000A3E6B0E0EC91FF27A5E6B0E091E0B7D169
:1007C0004091650000916000041709F401C036C033
:1007D00000C0A1E6B0E08C918F5F8C9308F452CEFC
:1007E00084D081D0E0ECFBE078D0969A8AEF8093B9
:1007F000640081E08093660042D00027BB27A0E31D
:100800008C9182FB0EF401E040E0041709F001C076
:10081000F4CF6BD0ECE3FBE060D065D0E2EDFBE021
:100820005CD0E1E0F0E072D0949AE2E0F0E06ED0CB
:100830009498E1E0F0E06AD058D0089556D0E0EE08
:10084000FBE04BD050D0ECE3FBE047D0969A8AE532
:100850008093640089E08093660011D00027BB2755
:10086000A0E38C9182FB0EF401E040E0041709F054
:1008700001C0F4CFE2E0F0E049D037D0089580E045
:10088000809361004091660000916100041710F0B0
:1008900009F013C0939AA4E6B0E08C919927B3D0E5
:1008A0009398A4E6B0E08C919927ADD0A1E6B0E092
:1008B0008C918F5F8C9308F4E5CF0895ED91FC91B6
:1008C000EF5FFF4FFC93EE930895A8E2B4E08D91A3
:1008D000882311F066D0FBCF0895A4D0802D11F0AD
:1008E00060D0FBCF089580EC62C081E060D014D06E
:1008F00080E85DC08FE7213039F08FEB223021F0A6
:100900008FE8233009F08FEC810F51C088EE93E01F
:100910007AD03197D9F7089583E0992774C08AEF88
:1009200090E071D0BD9ABC9ABB9ABA9AB99AB89A1B
:10093000C09885E090E067D0C198C598C498C39AE4
:10094000C29AC19AEF93FF93E5E1F0E050D0FF9196
:10095000EF91C19855D0C19AEF93FF93E5E1F0E094
:1009600046D0FF91EF91C1984BD0C19AEF93FF937E
:10097000E5E1F0E03CD0FF91EF91C19841D0C29801
:10098000C19AEF93FF93E5E1F0E031D0FF91EF9151
:10099000C19836D088E20BD08EE009D086E007D02F
:1009A0000895C09A829505D004D02AD00895C098A1
:1009B000F9CF859510F4C29A01C0C298859510F4BC
:1009C000C39A01C0C398859510F4C49A01C0C49815
:1009D000859510F4C59A01C0C598C19AEF93FF930D
:1009E000E5E1F0E004D0FF91EF91C19808953197CF
:1009F000F1F70895689462F80895E89462F808950C
:100A000081E090E000C0EF93FF93EE27E82BE92B05
:100A100031F0EAEFF0E03197F1F70197D1F7FF916C
:100A2000EF910895C895319600200895000F111F89
:100A3000221F331F089500951095209530950F5F64
:100A40001F4F2F4F3F4F0895019110810EC001910C
:100A50001191219130810BC00191108117FF05C0C8
:100A60003FEF2FEF04C0008111272227332737FFE4
:100A700003C0E1DF8DE28D93CF93DF93CF92DF92BE
:100A8000EF92AA24BB24CC24DD24EE2440E2CAE069
:100A9000DD2755E093E38881890F87FD9F7083FDF3
:100AA000907F891B89935A95A9F7C0DFAA1CBB1CAC
:100AB000CC1CDD1CEE1C4A9551F7E894EFE0FF27B3
:100AC00082910ED0EB30E0F71EF068948A2D0CD0A6
:100AD00088278D93EF90DF90CF90DF91CF9108958D
:100AE000982F829501D0892F8F70805D26F08033FA
:100AF00009F4089568948D930895E199FECFEEBBB3
:100B0000FFBB3196089591E001C092E07B3751F42C
:100B10007FB7F894F2DF8D918DBBE29AE19A9A95B6
:100B2000C9F77FBF7727089591E001C092E0E5DF24
:100B3000E09A8DB38D939A95D1F708955757572E14
:100B40004156522E344D472E434F4D0047534D3A98
:100B500000002B33383600003400300038003300FA
:100B600032003100370039002020496E73657274FD
:100B7000204361726420200043617264206E756DB1
:100B80006265723A0000436172642077726974741E
:100B9000656E000045726173696E6720436172641F
:100BA0007300202020436172647320657261736555
:100BB000640020202020436865636B696E67000035
:100BC00020436172642065786365707465642020D9
:100BD000000020202020556E6C6F636B6564000060
:0E0BE000202020436172642077726F6E6700E0
:00000001FF
